:020000040000FA
:100000000E200C3012200F3086016300860A06088D
:100010000F390F3A031D0528162000288316860184
:100020008312080083168100831208000D3012200D
:1000300005308D006300860163008D0B20280800C9
:060040000F3086001A28B3
:084000000100020003000400AE
:02400E00F53F7C
:104200002400490064003A00200063006F0075003C
:104210006E0074002E00610073006D002C007600AB
:10422000200031002E003900200032003000300024
:1042300032002F00300033002F003100300020000A
:10424000310035003A00340033003A0035003600C2
:104250002000740075006E00640072006100200090
:104260004500780070002000740075006E00640046
:0842700072006100200024002F
:00000001FF
